S013000050617573655377697463682E73726563A1
S11300000EC028C027C026C025C024C023C022C0DB
S113001021C020C04DC01EC01DC01CC01BC0112467
S11300201FBECFE5D2E0DEBFCDBF10E0A0E6B0E05A
S1130030E4E1F1E002C005900D92A236B107D9F7D0
S113004020E0A2E6B0E001C01D92A336B207E1F7BA
S113005006D05EC0D5CF86B380958170089588E1BF
S113006087BBB898C09A1ABC13BE12BE83B785600A
S113007083BF80E189BF7894C39AC1E0ECDF882311
S1130080E9F380916000813021F4C39810926000FC
S113009005C0811103C0C39AC09360002FEF84E3AD
S11300A09CE0215080409040E1F700C00000E6CF82
S11300B01F920F920FB60F9211248F9380916000BC
S11300C0811102C0C49A1EC08130E1F480916200A3
S11300D08F3099F480916100813021F4C49810929A
S11300E0610008C080916100811104C0C49A81E05C
S11300F0809361001092620005C0809162008F5F5E
S1130100809362008F910F900FBE0F901F901895EF
S1070110F894FFCF8D
S10501140101E3
S9030000FC
